:1030000055C000006EC000006CC000006AC0000027
:1030100068C0000066C0000064C0000062C000001C
:1030200060C000005EC00000E2C300005AC00000A3
:1030300058C0000056C0000054C0000052C000003C
:1030400050C000004EC000004CC000004AC000004C
:10305000E5C1000046C0000044C0000042C00000BE
:1030600040C000003EC000003CC000003AC000006C
:1030700038C0000036C0000034C0000032C000007C
:1030800030C000002EC000002CC000002AC000008C
:1030900028C0000026C0000024C0000022C000009C
:1030A00020C000001EC000001CC0000011241FBE74
:1030B000CFEFD5E0DEBFCDBF11E0A0E0B1E0EAE1A7
:1030C000FEE302C005900D92A63DB107D9F721E0BD
:1030D000A6EDB1E001C01D92A43FB207E1F72FD0E9
:1030E0009AC68ECF8091D601882341F18091E60166
:1030F0009091E701A091E801B091E90180784091B9
:10310000DE015091DF016091E0017091E10148170B
:1031100059076A077B0791F025E0FA0120935700D1
:10312000E89507B600FCFDCF8093DE019093DF01A8
:10313000A093E001B093E1011092D601089584B705
:10314000877F84BF88E10FB6F89480936000109267
:1031500060000FBE90E080E80FB6F89480936100A5
:10316000909361000FBEC1E0C5BF82E085BF22D34E
:10317000C0936F0083E080938100789411E043E076
:10318000E42E01E054E0D52E66E0C62E73E0B72EA3
:10319000E2E0AE2E80910001882309F428C181E08D
:1031A00091E07FD5F82E882309F41CC1C0E0D0E05F
:1031B000FC1609F417C181E091E097D59091D701F1
:1031C000992311F08A33D1F41092DD014090E2018D
:1031D0005090E3016090E4017090E5014092E601B7
:1031E0005092E7016092E8017092E9011092DA01D1
:1031F0008A3309F0F5C00093D701F2C02FEB280FF6
:10320000263010F4875304C080538A3008F0E8C099
:103210002091D90140E1249F90011124282B209373
:10322000D9018091DA0181278093DA018111D8C018
:103230008091DD01963009F4C2C0820F8093DD01D8
:10324000933059F100F5913019F1923009F0C6C070
:10325000422F50E0542F44278091E6019091E701DE
:10326000A091E801B091E901840F951FA11DB11D46
:103270008093E6019093E701A093E801B093E90100
:10328000B092D701ADC09430F9F0953049F1A6C0A5
:103290002093DC01A092D701A3C04090E60150909A
:1032A000E7016090E8017090E901420E511C611C39
:1032B000711C4092E6015092E7016092E801709221
:1032C000E901D092D7018CC02093DB018091DC0111
:1032D000882311F085E001C086E08093D70180C08B
:1032E0008091DC0181508093DC014090E601509098
:1032F000E7016090E8017090E901411490E35906FC
:103300006104710428F01092D7011092D60168C0B0
:1033100080FF03C02093D80163C0422F50E0542F98
:1033200044278091D801482B8091DB01823049F1FC
:10333000843089F181113CC08091D60181110CC08B
:10334000E091DE01F091DF01E0925700E89507B6C9
:1033500000FCFDCF0093D601F2010A011093570043
:10336000E8951124F2E04F0E511C611C711C409233
:10337000E6015092E7016092E8017092E901B2DE45
:1033800017C060E070E094E0440F551F661F771F80
:103390009A95D1F705C060E070E0BA01552744273F
:1033A0004093E2015093E3016093E4017093E501DF
:1033B0008091DC01811114C0C092D70111C0422F4D
:1033C00050E0819590E04817590751F48BDE8091C9
:1033D000DB01813029F41092000102C01092D70164
:1033E0002196E6CE81E091E00FD4B4D3D3CE809184
:1033F000E00081608093E00082E49CED9093F50111
:103400008093F4012CE088E190E00FB6F894A89541
:10341000809360000FBE20936000FFCF1F920F9239
:103420000FB60F9211240F900FBE0F901F9018959A
:103430000895089581E091E0A8D31092D7010895EE
:1034400081E091E07FC4292F33272230310559F0E4
:103450002330310569F021303105D9F482E190E063
:1034600029E831E01AC080E290E029E631E015C099
:1034700099278330910568F4FC01EE0FFF1FED5E84
:10348000FE4F20813181FC01E05FFE4F808190E0A2
:1034900004C080E090E020E030E0FA013183208336
:1034A000089507B600FCFDCFF999FECF23E0FB019C
:1034B00020935700E89507B600FCFDCF81E180938B
:1034C0005700E895089507B600FCFDCFF999FECFA7
:1034D00025E0FB0120935700E89507B600FCFDCFDF
:1034E00081E180935700E895089507B600FCFDCF71
:1034F000F999FECF21E0FB010A0120935700E895DE
:103500001124089521E2FC0120935700849108952D
:1035100029E0FC012093570084910895E1E0F0E058
:1035200089E0809357008491089507B600FCFDCF91
:10353000F999FECF809599E0E1E0F0E0082E9093B4
:103540005700E89508952091F2013091F301261774
:10355000370748F06115710539F42091E8002E779E
:103560002093E80001C0B901FC0120E0611571055C
:10357000A1F18EB38823F1F18530F1F18091E8005B
:1035800083FD3CC08091E80082FF06C08091E80086
:1035900082FF26C080E008958091E80080FFE6CF9A
:1035A0002091F3008091F20090E0922B611571055B
:1035B00051F08830910538F421912093F100615049
:1035C00071090196F3CF21E0089709F020E080917E
:1035D000E8008E778093E800C9CF2111CACFD6CFFB
:1035E0008EB3882339F0853039F08091E80083FF6D
:1035F000CDCF04C082E0089583E0089581E008956E
:103600008F708093E900EBEEF0E080818160808331
:10361000EDEEF0E010826093EC0040838091EE00CC
:10362000881F8827881F08950F931F93CF93DF93D8
:10363000062FEC0110E0101771F19881992341F1E8
:103640002C81E981FA817B81892F8F70873010F07E
:1036500080E022C0223010F056E001C052E028E0A5
:1036600030E040E02E173F0720F44F5F220F331F5A
:10367000F9CF4295407F452B692F661F6627661F4D
:1036800090E4799F90011124622BBADF882301F323
:103690001F5F2596D0CF81E0DF91CF911F910F91D1
:1036A00008958091EC0187FD05C08091E80080FFBE
:1036B0000DC010C08091E80082FD04C08EB381115E
:1036C000F9CF08958091E8008B7707C08EB3811100
:1036D000ECCF08958091E8008E778093E8000895FC
:1036E0008091E4009091E50045E62091EC0020FFF8
:1036F00020C02091E80020FD20C02EB3222389F0B5
:10370000253089F02091EB0025FD0FC02091E400C9
:103710003091E5002817390741F3415041F0C901C4
:10372000E4CF82E0089583E0089581E0089584E085
:1037300008952091E80022FFE0CF80E008950F93E4
:103740001F93CF93DF9346D04DD0C8EDD0E0888152
:103750008F77888388818068888388818F7D88833C
:1037600019BC1EBA1092EA0100EE10E0F801808147
:103770008B7F808388818160888342E060E080E085
:103780003FDFE1EEF0E080818E7F8083E2EEF0E0CB
:10379000808181608083808188608083F80180815E
:1037A0008E7F8083888180618883DF91CF911F9194
:1037B0000F910895E8EDF0E080818F7E8083E7ED42
:1037C000F0E080818160808384E082BF81E080932B
:1037D000EB01B5CFE8EDF0E080818E7F8083109221
:1037E000E20008951092DA001092E10008951F920D
:1037F0000F920FB60F9211242F933F934F935F9325
:103800006F937F938F939F93AF93BF93EF93FF93A8
:103810008091DA0080FF19C08091D80080FF15C028
:103820008091DA008E7F8093DA008091D90019BCF4
:1038300080FF09C082E089BD09B400FEFDCF81E0B0
:103840008EBBF6DD02C01EBAF4DD8091E10080FF80
:1038500017C08091E20080FF13C08091E2008E7F4C
:103860008093E2008091E20080618093E200809189
:10387000D80080628093D80019BC85E08EBB69D1E6
:103880008091E10084FF2DC08091E20084FF29C077
:1038900019BC82E089BD09B400FEFDCF8091D8003B
:1038A0008F7D8093D8008091E1008F7E8093E1002E
:1038B0008091E2008F7E8093E2008091E20081603F
:1038C0008093E2008091EA01882311F084E007C030
:1038D0008091E30087FF02C083E001C081E08EBBDE
:1038E00038D18091E10083FF21C08091E20083FF05
:1038F0001DC08091E100877F8093E10082E08EBB54
:103900001092EA018091E1008E7F8093E100809126
:10391000E2008E7F8093E2008091E20080618093DC
:10392000E20042E060E080E06BDE13D1FF91EF91B6
:10393000BF91AF919F918F917F916F915F914F91C7
:103940003F912F910F900FBE0F901F9018951F93CE
:10395000CF93DF9300D0CDB7DEB7ECEEF1E08091EE
:10396000F100819381E0E43FF807C9F769DD8091B8
:10397000E80083FFDAC09091EC018091ED01853081
:1039800009F465C030F4813059F168F0833041F1B9
:10399000CCC0883009F49CC0893009F4ABC08630B3
:1039A00009F0C3C075C0903881F0923809F0BDC0ED
:1039B0008091F0018F708093E9009091EB0095FB6E
:1039C000992790F91092E90001C090E08091E800F9
:1039D000877F8093E8009093F1001092F10083C0FC
:1039E000292F2D7F09F0A1C0923009F09EC090913F
:1039F000EE01911126C02091F0012F7009F495C0BD
:103A00002093E9009091EB0090FF1BC0833021F4DC
:103A10008091EB00806213C08091EB008061809305
:103A2000EB0081E090E0022E01C0880F0A94EAF7D3
:103A30008093EA001092EA008091EB008860809306
:103A4000EB001092E9008091E800877F4FC0911150
:103A50006CC01091EE011F778091E3008078812B7C
:103A60008093E3008091E800877F8093E80019DE6F
:103A70008091E80080FFFCCF8091E3008068809314
:103A8000E300112311F083E001C082E08EBB4DC042
:103A90009058923008F049C0AE014F5F5F4F60917F
:103AA000F0018091EE019091EF01CDDC009709F4D7
:103AB0003CC02091E800277F2093E800BC01898169
:103AC0009A8141DD8091E8008B778093E8002DC0DA
:103AD000903859F58091E800877F8093E8008091C5
:103AE000EA018093F1008091E8008E778093E800EE
:103AF000D8DD1BC0911119C09091EE019230A8F44D
:103B00008091E800877F8093E8009093EA01C9DD07
:103B10008091EA01811104C08091E30087FF02C017
:103B200084E001C081E08EBB85DC8091E80083FFEA
:103B30000AC08091E800877F8093E8008091EB00C5
:103B400080628093EB000F900F90DF91CF911F91D7
:103B500008950895CF938EB38823A9F08091E9004A
:103B60008F709091EC0090FF02C090E801C090E04F
:103B7000C92FC82B1092E9008091E80083FDE7DE91
:103B8000CF70C093E900CF910895CF93DF93EC01FC
:103B90001E861D8688E18D8782E08C83898761E09F
:103BA000CE01019641DD882331F061E0CE01069619
:103BB000DF91CF9139CD80E0DF91CF9108952EB381
:103BC000243001F5FC0181818F708093E900209100
:103BD000F3008091F20090E0922B892B89F0909174
:103BE000E8008091E8008E778093E80095FD08C09A
:103BF00077DD811108C08091E8008E778093E8001E
:103C000080E0089582E00895CF93DF93EC018EB3B6
:103C1000843009F043C089818F708093E9008091DE
:103C2000E80080FF02C0CE01CADF8E858823B1F193
:103C30002E812F7081E090E0AC0102C0440F551F2F
:103C40002A95E2F74093EA001092EA0029812F704A
:103C5000022E01C0880F0A94EAF78093EA001092BE
:103C6000EA008E818F708093E9008091EB00806183
:103C70008093EB008091EB0088608093EB0089815A
:103C80008F708093E9008091EB0080618093EB005E
:103C90008091EB0088608093EB001E86DF91CF91CE
:103CA00008952EB3243019F080E090E00895FC01CF
:103CB00086818F708093E9008091E80082FFF4CFC5
:103CC0002091F3008091F20090E0922B009731F464
:103CD0002091E8002B772093E80008952091F300CD
:103CE0008091F20090E0922B08952EB3243019F0C9
:103CF0008FEF9FEF0895FC0186818F708093E9001C
:103D00008091E80082FFF4CF2091F3008091F200CF
:103D100090E0922B892B21F02091F10030E002C03D
:103D20002FEF3FEF4091F3008091F20090E0942B51
:103D3000892B29F48091E8008B778093E800C901F2
:103D400008950895CF93DF93EC018091E80083FFFD
:103D50005FC0888190E02091F0013091F101281737
:103D6000390709F055C08091ED01813051F120F003
:103D7000823009F43DC04CC08091EC01813A09F0D9
:103D800047C08091E800877F8093E8008091E80039
:103D900080FD04C08EB38111F9CF3AC0EB85FC855C
:103DA000DF010D900020E9F7BD01615071096E1B24
:103DB0007F0B7093F1006093F1008B859C85C3DBD2
:103DC00014C08091EC01813A19F58091E800877F59
:103DD0008093E8008091E80080FD04C08EB38111DB
:103DE000F9CF16C08D858093F100DF91CF9159CC2A
:103DF0008091EC01813261F48091E800877F8093AB
:103E0000E8004FDC81E08E87CE01DF91CF9199CF22
:0A3E1000DF91CF910895F894FFCFE1
:103E1A000100834000000104400000019B010000F2
:103E2A0004183065014B01190130034C0055004656
:103E3A0000410020005000720069006E00740065A5
:103E4A00007200200042006F006F0074006C006F67
:103E5A0000610064006500720000001803440065F8
:103E6A000061006E002000430061006D0065007271
:103E7A000061000000040309040902200001010096
:103E8A00803209040000020701020007058302408C
:103E9A000005070504024000051201100100000098
:103EAA0008EB036B200100010200014D46473A4727
:103EBA00656E657269633B4D444C3A47656E65723F
:103ECA0069635F2F5F546578745F4F6E6C793B430B
:103EDA004D443A313238342E343B434C533A5052E3
:063EEA00494E5445520050
:103FA00080CA91CAA2CAAECAB3CAB8CABECA089564
:083FB000089508950895089595
:103FE000DFCFDFCFDFCFDFCFDFCFDFCFDFCFDFCF61
:083FF000DFCFDFCFDFCFDFCF11
:083FF8000030000020DFFBDCBB
:0400000300003000C9
:00000001FF
